:100000006F00605C1300000013000000130000008C
:100010001300000013000000130000001300000094
:100020001300000013000000130000001300000084
:08003000130000007300100032
:100038000000000000000000080300000C0300009E
:10004800000000000C050000000000000000000097
:100058000E05000010050000000000000000000070
:100068001205000000000000140500000000000058
:1000780016050000180500001A0500001C05000000
:100088001E050000200500002205000024050000D0
:1000980026050000280500002A0500002C050000A0
:1000A8002E05000030050000320500003405000070
:1000B80036050000380500003A0500003C05000040
:1000C8003E05000040050000420500004405000010
:1000D80046050000480500004A0500004C050000E0
:1000E8004E050000500500005205000054050000B0
:1000F80056050000580500005A0500005C05000080
:100108005E0500006005000062050000640500004F
:1001180066050000680500006A0500006C0500001F
:100128006E050000700500007205000074050000EF
:1001380076050000780500007A0500007C050000BF
:100148007E0500008005000082050000840500008F
:1001580086050000880500008A0500008C0500005F
:100168008E0500009005000092050000940500002F
:1001780096050000980500009A0500009C050000FF
:100188009E050000A0050000A2050000A4050000CF
:10019800A6050000A8050000AA050000AC0500009F
:1001A800AE050000B0050000B2050000B40500006F
:1001B800B6050000B8050000BA050000BC0500003F
:1001C800BE050000C0050000C2050000C40500000F
:1001D8000000000000000000000000000000000017
:1001E8000000000000000000000000000000000007
:0801F8000000000000000000FF
:10020000397101436EC619A0397141536AC866CA73
:1002100062CC5ECE19A0397101535AD056D252D455
:100220004ED64AD826DA22DC06DE330161408282CD
:1002300041114AC026C222C406C68282B24D410183
:10024000024D924C224CB24B4101024B924A224A3F
:10025000B2494101024992442244B24041018280A4
:100260003D432A876373C3029377F700BDEFADE583
:10027000937606FF3D8ABA960CC34CC30CC74CC795
:100280004107E36BD7FE11E28280B306C3408A06C2
:100290009702000096966780A6002307B700A30682
:1002A000B7002306B700A305B7002305B700A304D2
:1002B000B7002304B700A303B7002303B700A302CA
:1002C000B7002302B700A301B7002301B700A300C2
:1002D000B7002300B700828093F5F50F9396850051
:1002E000D58D93960501D58D61B79396270097021A
:1002F000000096968682E78086FA9680C1171D8F49
:100300003E96E374C3F8A5B77300203001A0EFF266
:100310003FF209451921152AB52D716513050520F0
:10032000792DB707002083A507083725000013059E
:1003300045C23D2F312EAA8537250000130545C340
:10034000052F37250000130545C4EF00B00301A0B9
:10035000B71702409843B706FFF84111136717001B
:1003600098C3D84337060200758FD8C39843B706A1
:10037000F7FEFD16758F98C39843B706FCFFFD1670
:10038000758F98C3D843B70681FFFD16758FD8C304
:100390009843B70600ECFD16758F98C33707FF002A
:1003A00098C723A6070202C402C69843C166558FA8
:1003B00098C3B716024005679C42F18F3EC6A2471C
:1003C00085073EC4B24781E7A247E397E7FEB71728
:1003D00002409C431397E7006357070685473EC6D4
:1003E00032478547631FF704B7170240D843B70663
:1003F000C1FFFD16D8C3D843D8C3D84313670740FD
:10040000D8C3D843758FD8C3D843B7062900558FB2
:10041000D8C39843B7060001558F98C398439316E5
:100420006700E3DD06FED843B7160240719BD8C3D0
:10043000D84313672700D8C32147DC42B18BE39E22
:10044000E7FE4101828002C661BF371602405C426E
:10045000370700209146B18B130707086385D70043
:10046000A1466388D702B7177A00938707201CC379
:10047000B7170240DC43918393F6F700B7070020DB
:1004800093870700B69794231C43B3D7D7001CC3A8
:10049000828054425042C167C982BD8A7D8E938753
:1004A000260085CABD466389D702C1466389D70243
:1004B000C54581466393B700C1470DE63746024004
:1004C00003260680418A15C637167A0013060620D1
:1004D0002DA08146C947D5B78546B547F9BF8146A6
:1004E000BD47E1BF3716024050429315E600E3DDF9
:1004F00005FC37163D0013060690B387C7021CC3E0
:10050000A5DA1C438583A5B701A001A001A001A025
:1005100001A001A001A001A001A001A001A001A0D3
:1005200001A001A001A001A001A001A001A001A0C3
:1005300001A001A001A001A001A001A001A001A0B3
:1005400001A001A001A001A001A001A001A001A0A3
:1005500001A001A001A001A001A001A001A001A093
:1005600001A001A001A001A001A001A001A001A083
:1005700001A001A001A001A001A001A001A001A073
:1005800001A001A001A001A001A001A001A001A063
:1005900001A001A001A001A001A001A001A001A053
:1005A00001A001A001A001A001A001A001A001A043
:1005B00001A001A001A001A001A001A001A001A033
:1005C00001A001A001A0970100209381A12B178118
:1005D0000020130121A317150000130525729705AC
:1005E0000020938525A21386818163FAC5008322AA
:1005F000050023A0550011059105E3EAC5FE13850A
:1006000081819385C1826377B500232005001105A0
:10061000E36DB5FEFD42739002BCAD427390428023
:10062000B76200009382820873A002309702000034
:100630009382C2A093E2320073905230EFF05FD108
:10064000970200009382E2CC739012347300203042
:10065000B7F7FF1F03A5477082809C4513F707017A
:1006600013F8F70001C7D8413368E8008E2113F76B
:10067000F50F39C318418146854E3D4F930F8002D7
:1006800093028004214E3396DE00B3F8C500631157
:1006900016039398260033131F011343F3FF337798
:1006A000E300B318180133E7E800639FF70550C96A
:1006B0008506E39AC6FD18C11307F00F6375B704EA
:1006C00054412146854E3D4F930F80029302800492
:1006D000414EB398CE0033F715016392E802131729
:1006E000260001173313EF001343F3FFB376D30053
:1006F0003317E800D98E639DF701232A15010506FB
:10070000E319C6FD54C18280E39457FA10C94DB76E
:10071000E39757FE23281501DDB723ACA180828023
:10072000371702405C439146B18B6385D700A146E1
:100730006382D706B7177A00938707201CC1371644
:1007400002405C4237070020130707019183BD8BED
:10075000BA9794231C41B3D7D7005CC15442A182FD
:100760009D8ABA969422B3D6D70014C55442AD825E
:100770009D8A36971823B3D7E7005CC55842398362
:10078000937637001387418036971823B3D7E70253
:100790001CC982805C435843C166C983758FB7F614
:1007A000FF1F83A6C670BD8B890713961601634889
:1007B0000600C54601466392D702C94739A8894653
:1007C000638FD702BD46638ED702C146638ED702C0
:1007D000C54601466393D700C1471DEF3747024026
:1007E00003270780418B05C737177A0013070720B7
:1007F000B307F7021CC121D61C41858381B701468E
:100800006DBF0546B547D1BF0146BD47F9B737179C
:100810003D0013070790E9BFB7150240D85593165E
:10082000F700D85563DF060411833D8B930617004C
:1008300037177A00130707203357D70218C1D4554A
:10084000A182BD8A8DE295463307D702058318C180
:1008500037170240585714413D8B050733D7E6023E
:1008600018C1184171B785456394B600E546E9BFE4
:10087000BD456396B600D1463387E602C9BF8906F7
:10088000E5BF3D8B9306170037177A001307072043
:100890003357D702F1B799C5371702401C4F5D8D0A
:1008A00008CF8280B7170240984F1345F5FF798D26
:1008B00088CF8280EFF2DF971629F577FD17F58F45
:1008C000F621DA257971D58F1EA95625FD779387F4
:1008D000379FF58FD6212A842EC6D58F9625D58FA2
:1008E000B625D58F5EA55E29C207C18393F7F7CFE2
:1008F000D98F5EA968082D35B747014093870780D7
:10090000B2456319F404A25756246547B387E7023A
:10091000C206C186984163D10604060752244206E6
:10092000B3D7E702130740064186B3D6E702B3F711
:10093000E7029206635406028E0793872703B3D714
:10094000E70213F77700B367D700C207C1831EA47D
:10095000456109B292574DBF0A07C9B792079387FD
:100960002703B3D7E702BD8BD58FC5B791C55E25E9
:100970000967D98F5EA582805A25F977FD17F98F0F
:10098000D5BF93F5F51F4EA182800A216D8D3335B9
:10099000A0008280B707002083A7070837177A00D6
:1009A00013070720B3D7E70293F7F70F238FF180E0
:1009B0001307803EB387E702239EF1808280EFF227
:1009C0003F872A841165011185451105E935930793
:1009D00000207C82371501408D473EC44C00E14722
:1009E000130505803EC6953922C837440140B70734
:1009F00008000C08130504803ECC02CA231E010027
:100A0000553D854513050480953705616FF09F843A
:100A1000EFF27F80B7440140AE893289014493846C
:100A20000480634524014A856FF03F8293050004EA
:100A30002685A13F65DDB38789008385070026856C
:100A40000504C205C181353FE9BF138781801C437E
:100A50009386C1823E95636BD500B786002093864E
:100A6000068063E5A60008C33E858280FD57EDBF82
:100A700039713EDA2ED232D436D63AD842DC46DE4E
:100A80009387C18022CC804326CA06CEAA8409C49B
:100A90001C4C99E32285ED290C44541026862285AE
:100AA00036C6EF007012F2406244D2442161828067
:100AB000011126CA4AC806CE22CC4EC652C4AA8408
:100AC0002E8901C51C4D91E3E1219C4C804499E3A2
:100AD00026857D29971700009387871A631BF402E8
:100AE000C0405E24A18BB1C71C48A1C7FD59294A4B
:100AF0001C4483450900FD17B1E91CC463DD0706EA
:100B00002286A94526856120FD576308F5022945FF
:100B100035A0971700009387A7186314F40080444A
:100B2000C9B7971700009387A713E31CF4FAC044D2
:100B30004DBFA2852685112A55D97D55F2406244C4
:100B4000D2444249B249224A056182801CC4050947
:100B500063D70700184C63CAE700638845011C404F
:100B60001387170018C08CA361B72286268505203D
:100B7000E31035F9D9B71C401387170018C029476F
:100B800098A371B79387C180AA85884315B70111CF
:100B900022CC26CA4AC806CE4EC6AA842E893284E2
:100BA00001C51C4D91E3ED26971700009387470D73
:100BB0006317F406C0401C4C1CC45E24A18BC1C347
:100BC0001C48B5CF1C4808409379F90F1379F90FE9
:100BD0001D8D5C486346F500A2852685692C25E5B8
:100BE0001C440505FD171CC41C401387170018C0C2
:100BF000238037015C486388A7005E24858B81CB06
:100C0000A9476316F900A2852685B5240DEDF240AB
:100C100062444A85D2444249B249056182809717AD
:100C200000009387E7076314F400804469B79717BF
:100C300000009387E702E310F4F8C044ADBFA2853B
:100C40002685212041D17D59D9B741119387C18093
:100C500026C2844322C44AC006C62A892E8489C477
:100C60009C4C99E326852D26971700009387470112
:100C7000631BF402C0400317C40093170701C1832C
:100C800093F68700ADEA93F6070195EEA54723207A
:100C9000F900136707045AA47D55B24022449244D8
:100CA00002494101828097170000938767FF631410
:100CB000F4008044C9B797170000938767FAE31CD4
:100CC000F4FAC0444DBF918B9DC34C5889C993071A
:100CD00044046384F5004A853123232A04025E24F8
:100CE0002322040093F7B7FD5EA41C481CC05E24B9
:100CF00093E787005EA41C4899EB5E24130700204D
:100D000093F707286385E700A2854A85A1215E2421
:100D100013F717001DC35C4823240400B307F040F9
:100D20001CCC1C480145B5FB8317C40013F707080A
:100D30002DD793E707045EA485B7898B014791E31C
:100D4000584818C4F9BFDE25011122CC26CA06CEA8
:100D50004AC84EC613F78700AA842E8479EBD8417F
:100D6000634DE000B841634AE0000145F24062444F
:100D7000D2444249B2490561828058547DD703A9C3
:100D800004009396370123A0040063DB0606704835
:100D90005E24918B99C75C401D8E5C5899C33C4082
:100DA0001D8E5C540C50814626858297FD575A242F
:100DB000631DF5009440F54763E8D706B707402068
:100DC0008507B3D7D700858BA5C31C482322040011
:100DD0001CC09317370163D80700FD576314F50053
:100DE0009C4091E368C84C5823A02401BDDD9307C3
:100DF00044046384F5002685F526232A0402B5B74A
:100E00000C500146854626850297FD572A86E31138
:100E1000F5F89C40B5DF75476385E7005947639354
:100E2000E70423A0240191B7136707045AA47D5552
:100E300035BF83A90501E38A09F203A905008D8B5B
:100E400023A0350133093941014791E3D84918C43A
:100E5000E35D20F11C540C50CA864E86268582978D
:100E60006347A0005E2493E707045EA4C9B7AA996C
:100E70003309A940F1BF9C49B9CF011122CC06CE5C
:100E80002A8411C51C4D81E72EC61922B245971739
:100E900000009387E7DE639BF5004C408397C50015
:100EA00095C722856244F240056171BD9717000025
:100EB000938707DF6394F5000C44CDB797170000C4
:100EC000938707DAE39CF5FC4C44C9BFF2406244C7
:100ED00001450561828001458280411122C406C618
:100EE0002A844EA572A52320050023220500232471
:100EF00005002322050623280500232A0500232CAC
:100F00000500214681451305C505EFF06FB597171C
:100F10000000938747B15CD097170000938767B3B1
:100F20001CD497170000938747B75CD4971700002D
:100F30009387A7B900D01CD8B240224441018280D7
:100F400097050000938565F3A9A2411126C21306F7
:100F500080069384F5FFB384C4024AC02E8922C45C
:100F600006C6938544071D262A8401CD232005004B
:100F700023222501310508C4138684068145EFF03C
:100F80002FAE2285B2402244924402494101828020
:100F90001C4DADE3411106C622C49707000093879C
:100FA00067FA1CD5938701819C43232405042326DB
:100FB0000504232805046314F50085471CCD2A8405
:100FC0001D2848C02285052808C422852D2048C434
:100FD000484001469145113708440546A545F53D71
:100FE00048440946C945D53D85471CCCB2402244FA
:100FF00041018280828041119387018126C284430E
:101000004AC006C69C4C22C42A8999E326854937E2
:10101000938484048044DC40FD1763D607009C4021
:10102000B9CF8440C5BF0317C40039E7C17785072E
:101030002322040623200400232204002324040086
:101040005CC423280400232A0400232C0400214626
:1010500081451305C405EFF0AFA0232A0402232C19
:10106000040223240404232604042285B2402244DB
:1010700092440249410182801304840671BF914564
:101080004A85E13588C051FDB1472320F90001446C
:10109000E9BF797122D44AD052CC56CA5AC85EC62A
:1010A00006D626D24ECE2A8AAE8A1304850401497A
:1010B000054BFD5B09ECB25022544A85925402590B
:1010C000F249624AD24A424BB24B456182800444A3
:1010D00083294400FD1963D409000040E1BFDE24E8
:1010E000637BFB008397E40063877701A6855285C5
:1010F000829A3369A90093848406E9BF1971A6DA3C
:10110000AE848395E500A2DC86DE328463DB0500D5
:10111000DE2423A0060093F7070885E79307004025
:101120001DA0300836C6EF00D01FB246E34205FED0
:101130007247BD67F98F7977BA9793B717009CC24A
:10114000F1BF930700041CC0F6506654D654014505
:1011500009618280DE25011122CC06CE26CA4AC84A
:10116000898B2E8489CF930774041CC01CC88547C3
:101170005CC8F2406244D2444249056182807400F6
:101180003000AA84A53FA2452A892685012219E9B3
:101190008317C40013F7072069FFF19B93E727002B
:1011A0005EA4D1B7970700009387C7D99CD45E246B
:1011B00008C008C893E707085EA4A2475CC8B24706
:1011C00081CF8315E4002685EF00501811C55E24F9
:1011D000F19B93E717005EA45E243369F9002316A0
:1011E000240141BFDDC183A7C5FF411122C406C64A
:1011F00026C21384C5FF63D307003E94AA84EF0080
:10120000B01B938701829C4381EF2322040023A01B
:1012100081822244B2402685924441016F00F01938
:10122000637EF40014403307D4006396E7009843CC
:10123000DC43369718C05CC0D9BFBA87D84319C3FE
:10124000E37DE4FE94433386D700631F860010409D
:10125000B29694C33386D700E31DC7FA10435843B0
:10126000B29694C3D8C375B76375C400B1479CC028
:101270004DB71040B306C4006316D700144358435B
:10128000B29614C058C0C0C369B78280011126CA83
:1012900093843500F19806CE22CC4AC84EC6A104EC
:1012A000B14763F3F404B14463E2B4042A89EF0064
:1012B000B0109387018298433A8439E09387418242
:1012C0009C4391E781454A85052F23A2A182A685EB
:1012D0004A851D27FD5963193507B1472320F900B9
:1012E0004A85EF00900D29A0E3D004FCB1471CC152
:1012F0000145F2406244D2444249B24905618280CC
:101300001C40858F63CF0702AD4663F6F6001CC014
:101310003E9404C031A05C406313870223A0F18295
:101320004A85EF0090091305B400930744006199C2
:101330003307F5405DDF3A94898F1CC05DBF5CC305
:10134000C5B72287404095BF130435007198E3026A
:1013500085FCB305A4404A854525E31C35FBB5BF94
:101360001C46FD171CC663DA0700184E63C5E7006C
:10137000A9476394F5006FF09F811C422E85138767
:10138000170018C28CA38280011122CC26CA4AC839
:101390004EC652C406CE2A89AE893284B304D60022
:1013A0007D5A63149400014501A80C204E864A859D
:1013B000453F0504E31745FFF2406244D2444249E9
:1013C000B249224A05618280357122CD26CB4AC9B5
:1013D0004EC706CF52C556C35AC1DEDEE2DCE6DA9E
:1013E000AA89AE843289368401C51C4D91E34D36FD
:1013F000971700009387C7886397F40C83A449006C
:10140000DE24A18BFDC39C48EDC393070002A30417
:10141000F1029307000302D22305F10222C6930BC7
:101420005002971A0000938AAA89054C294B4A84D6
:101430001C2099C3639E770DB30C2441638D0C006F
:10144000E6864A86A6854E858137FD57630FF51CD3
:101450009256E69636D21C206389071CFD57130965
:10146000140002C802CE3ECA02CCA309010482D4F1
:101470008345090015465685252713041900C247E0
:1014800051E913F7070109C713070002A309E10493
:1014900013F7870009C71307B002A309E1048346C5
:1014A00009001307A002638FE606F2474A848146CB
:1014B0002546182093051400130707FD6377E60AF5
:1014C000B5CA3ECE85A8970700009387677D6395D0
:1014D000F40083A489002DB797070000938747780D
:1014E000E390F4F283A4C90021BFA6854E85EFF0F6
:1014F000CFF501DD7D55FA406A44DA444A49BA49DC
:101500002A4A9A4A0A4BF65B665CD65C0D61828079
:10151000050439BF330555413315AC00C98F3EC8AA
:101520002289B9B7324793064700184336C6634746
:1015300007023ACE18209307E002631DF704183023
:101540009307A002631BF702B24709041387470001
:101550009C433AC663C107023ECA2DA83307E04048
:1015600093E727003ACE3EC8F1B7B38767038546B5
:101570002E84BA973DBFFD57C5B7050402CA814600
:1015800081472546182093051400130707FD63744F
:10159000E606F9F20C200D46170500001305C5728A
:1015A000012511CD97070000938707721D8D9307C2
:1015B0000004B397A700424505045D8D2AC80C209E
:1015C000194617050000130565701309140023045C
:1015D000B102F92335C197F7FFFF9387A7A295E7DB
:1015E0004247B2471377071009CF91073EC692577B
:1015F000D2973ED22DBDB387670385462E84BA9716
:1016000051B79D07E19BA107D5B778009706000069
:101610009386C6D726860C084E8597000000E70003
:101620000000FD572A8AE314F5FCDE2493F7070433
:10163000E39207EC1255C1B5780097060000938637
:10164000E6D426860C084E85012AE1BF797156CA78
:101650009C49BA8A984522D426D24ECE52CC06D680
:101660004AD05AC85EC6AA892E84B284368A63D309
:10167000E700BA879CC00347340419C385079CC0A0
:101680001C4093F7070281C79C4089079CC003292F
:10169000040013796900631A0900130B9401FD5BC0
:1016A0005C449840998F634CF9041C408346340491
:1016B00093F70702B336D000A5EB13063404D285A6
:1016C0004E85829AFD576303F5041C4011469840ED
:1016D000998B544481446397C700B384E64063D335
:1016E000040081441C4418486354F700998FBE9449
:1016F000014969047D5B63982405014509A8854675
:101700005A86D2854E85829A631E75017D55B250E8
:10171000225492540259F249624AD24A424BB24B85
:10172000456182800509ADBF3307D400130600036D
:10173000A301C7040347540493871600A2978906A0
:10174000A381E7049DBF85462286D2854E85829A75
:10175000E30E65FB050945B7797122D426D24AD03C
:101760004ECE06D652CC56CA5AC8B689942D930787
:1017700090063289AA842E8413863504638DF6027E
:1017800063E2D706930780056385F61863EDD700FB
:10179000638D062093073004638EF60A930A2404AF
:1017A0002301D404C9A0930730066385F60A930782
:1017B0004006E395F6FE1C40084393F607089305A0
:1017C0004500C5C61C410CC363D807001307D002EF
:1017D000B307F040A301E404970600009386864F08
:1017E000294765A8930700076381F61663E5D702CA
:1017F0009307E0066388F6189307F006E390F6FA7D
:101800000C401C4313F805081385470063070806BE
:1018100008C39C4385A893075007E383F6FE93070C
:1018200080076388F61293073007E399F6F61C43A6
:10183000D04181459386470014C383AA070056858B
:10184000852601C53305554148C05C401CC8A3012D
:10185000040461A81C43930A2404938647009C4314
:1018600014C32301F4048547D5B793F607041C413C
:101870000CC3B9DAC207C18781BF93F5050408C359
:10188000C9D99E231307F0066386E60E970600006B
:10189000938646442947A30104044C400CC463C505
:1018A000050008406D9908C099E3B28A89CDB28AD3
:1018B000B3F5E702FD1AB6958C212380BA00B3D5A3
:1018C000E70263FFE70AA147631EF7001C40858B10
:1018D00091CB58401C4863C7E70093070003A38FD0
:1018E000FAFEFD1A3306564110C84E87CA867000AC
:1018F000A2852685A13B7D5A631D450B7D55B250BF
:10190000225492540259F249624AD24A424B4561EA
:101910008280A382D504970600009386A63B0C40E4
:10192000084313F805081C411105630D080208C39C
:1019300013F7150001C793E505020CC04147A1FF4D
:101940000C4093F5F5FD0CC0B9B79C4193E7070235
:101950009CC193078007A302F404970600009386B6
:10196000A63875BF13F8050408C3E30308FCC207D3
:10197000C1837DBF970600009386C635214721BFEE
:10198000AE873DB794411C43CC4913F80608138534
:1019900047006306080008C39C438CC339A008C3F2
:1019A00093F606049C43F5DA8EA323280400B28A3A
:1019B0002DBF14485686CA8526858299E30045F5D1
:1019C0001C40898B8DE7B2474844E35AF5F23E85C7
:1019D0003DB785465686CA8526858299E30065F31C
:1019E000050A5C443247998FE345FAFEE9BF014A94
:1019F000930A94017D5BF5B7411122C42A842E8598
:101A000023A4018206C6EFF04F84FD576317F5004B
:101A1000938781829C4391C31CC0B2402244410100
:101A20008280411122C42E848395E50006C6792266
:101A3000634905007C48AA977CC8B2402244410112
:101A400082805E247D777D17F98F5EA4FDB7DE2549
:101A5000011122CC26CA4AC84EC606CE93F70710FB
:101A6000AA842E843289B68991C78395E500894678
:101A7000014609225E247D777D17F98F5EA48315C8
:101A8000E4006244F240CE864A86B2494249268545
:101A9000D244056125A8411122C42E848395E50016
:101AA00006C6C928FD575A24631AF500FD77FD17AD
:101AB000F98F5EA4B2402244410182808567D98FAC
:101AC0005EA468C8C5BF8395E50005A8411122C47E
:101AD0002A842E85B285368623A4018206C6EFE0CD
:101AE0003FF3FD576317F500938781829C4391C3B1
:101AF0001CC0B240224441018280411122C42A8488
:101B00002E8523A4018206C6C520FD576317F50064
:101B1000938781829C4391C31CC0B24022444101FF
:101B20008280411122C42A842E85B28523A4018299
:101B300006C6C920FD576317F500938781829C4331
:101B400091C31CC0B240224441018280411122C491
:101B50002A842E8523A4018206C65D20FD576317C3
:101B6000F500938781829C4391C31CC0B2402244FC
:101B700041018280411122C42A842E85B285368695
:101B800023A4018206C65920FD576317F5009387E9
:101B900081829C4391C31CC0B24022444101828097
:101BA00093F5F50F2A966314C500014582801C2128
:101BB000E38EB7FE0505C5BF82808280411122C435
:101BC0002A842E85B285368623A4018206C6A920E2
:101BD000FD576317F500938781829C4391C31CC016
:101BE000B2402244410182809307800523A4F18200
:101BF0007D5582809307800523A4F1827D558280E4
:101C00009307800523A4F182014582809307800514
:101C100023A4F1827D5582809307800523A4F1825D
:101C20007D55828053797374656D436C6B3A25647E
:101C30000D0A00004368697049443A253038780D30
:101C40000A00000054686973206973207072696E1D
:101C50007466206578616D706C650D000000000091
:101C60000000000000000000000000000000000074
:101C70000000000000000000000000000000000064
:101C80000000000000000000000000000000000054
:101C90000000000000000000000000000000000044
:101CA0000000000000000000000000000000000034
:101CB000000000000000000000000000232D302B79
:101CC00020000000686C4C006566674546470000D0
:101CD0003031323334353637383941424344454662
:101CE0000000000030313233343536373839616224
:081CF00063646566000000005A
:101CF80000000000000000000102030406070809B4
:101D08000000000001020304010203040607080999
:101D1800000000007C1C00009C1C00005C1C0000F3
:101D280000000000000000000000000000000000AB
:101D3800000000000000000000000000000000009B
:101D4800000000000000000000000000000000008B
:101D5800000000000000000000000000000000007B
:101D6800000000000000000000000000000000006B
:101D780000D8B80502040608AC00002020000020A6
:081D8800200000200000000013
:00000001FF
